S01900006F70656E626C745F73746D3332663039312E73726563FF
S3150800000000800020B91F0008092000080920000800
S3150800001000000000000000000000000000000000D2
S315080000200000000000000000000000000920000891
S31508000030000000000000000009200008050900086B
S3150800004009200008092000080920000809200008DE
S3150800005009200008092000080920000809200008CE
S3150800006009200008092000080920000809200008BE
S3150800007009200008092000080920000809200008AE
S31508000080092000080920000809200008092000089E
S31508000090092000080920000809200008092000088E
S315080000A0092000080920000809200008092000087E
S311080000B0092000080920000809200008A3
S315080000BC10B5064C2378002B07D1054B002B02D024
S315080000CC044800E000BF0123237010BDC8000020BF
S315080000DC0000000054200008044B10B5002B03D078
S315080000EC0349044800E000BF10BDC04600000000EC
S315080000FCCC00002054200008002243088B4274D3FD
S3150800010C03098B425FD3030A8B4244D3030B8B42FE
S3150800011C28D3030C8B420DD3FF22090212BA030C07
S3150800012C8B4202D31212090265D0030B8B4219D3E8
S3150800013C00E0090AC30B8B4201D3CB03C01A524108
S3150800014C830B8B4201D38B03C01A5241430B8B4250
S3150800015C01D34B03C01A5241030B8B4201D30B0339
S3150800016CC01A5241C30A8B4201D3CB02C01A524160
S3150800017C830A8B4201D38B02C01A5241430A8B4223
S3150800018C01D34B02C01A5241030A8B4201D30B020C
S3150800019CC01A5241CDD2C3098B4201D3CB01C01A26
S315080001AC524183098B4201D38B01C01A5241430930
S315080001BC8B4201D34B01C01A524103098B4201D31E
S315080001CC0B01C01A5241C3088B4201D3CB00C01A8B
S315080001DC524183088B4201D38B00C01A5241430803
S315080001EC8B4201D34B00C01A5241411A00D2014628
S315080001FC524110467047FFE701B5002000F006F89B
S3150800020C02BDC0460029F7D076E770477047C0464E
S3150800021C72B6704762B6704730B5184B184C002545
S3150800022C2360184B8BB02363174B20006363802322
S3150800023CDB02236180235B0363610C23A561636086
S3150800024CE56125626562A562E562A560E56000F078
S3150800025CEFFE0E4A012300920D4A079302920422DE
S3150800026C089369460D33200005950695019503926A
S3150800027C0495099300F064FE0BB030BD0064004091
S3150800028CE40000204C01002028010020E0CC0000EE
S3150800029CE0FF000003000D4810B5026B0C4C116111
S315080002AC146000249460D46000290AD00139C9B2BC
S315080002BC0131143259181C780133147001328B42EF
S315080002CCF9D1322100F062FF10BDC046E4000020CF
S315080002DCE1070000F8B5154C06000D0000220021B8
S315080002EC200001F05FF80023002805D1626B104945
S315080002FC176803008F4201D01800F8BD91680029D1
S3150800030CFAD11369002B0ED00023D218127D0133B3
S3150800031C3254626BDBB2116918008B42F5D3C9B241
S3150800032C29700123E8E70021FAE7C046E40000201B
S3150800033C6706000010B5FFF76BFF10BD70B582B0ED
S3150800034C00F084FA002801D102B070BD00F07EFDE1
S3150800035C0028F9D000F0EEFB00F09AFA00F0BCFD8C
S3150800036C0123114A80259169AD051943916192695A
S3150800037C13400193019B00F06DFA06000400C03689
S3150800038C2D1A23782B55013400F00AFCB442F8D107
S3150800039C0321064A13680B43136000F05BFA4468A2
S315080003ACFFF738FFA047CFE70010024000000140D6
S315080003BC70B5551EADB2002A0AD00C006D18013561
S315080003CC461A23783355013400F0EAFBAC42F8D1CF
S315080003DC70BDC046F0B5C6460F4B00B5070098462B
S315080003EC1D1D00260D4C01E0AC680C3500F0D8FB41
S315080003FCBC4204D82B689C466444A74206D30136F3
S3150800040C122EF1D1FF2004BC9046F0BD73009E1944
S3150800041CB6004644307AF6E76C2000080028000837
S3150800042CF8B5CE46474680B507000068FFF7D2FFF9
S3150800043C0024FF2824D001F02FF981239B0099462C
S3150800044C04235B42DB1B3D1DB944984605E0236833
S3150800045C9E4212D104354D4517D043465C193B686C
S3150800046C2E689C46644400F09BFB32000023210056
S3150800047C022001F057F90028E9D0002401F01EF9F2
S3150800048C20000CBC90469946F8BD0124F6E7C046F8
S3150800049C70B50F4C06000D00A04217D00D4B9942B3
S315080004AC09D0FFF7BDFF002801D0EB0502D00024C8
S315080004BC200070BD34002368AB42F9D0200080229E
S315080004CC20C092002900FFF773FFF1E7024EECE714
S315080004DC6C0300200028000868010020F0B5464689
S315080004ECD6464F46C0B51E004B0A5B029A460368B1
S315080004FC80460C0015005A1C38D09A4507D0404641
S3150800050C5146FFF7C5FF804600282DD003680434F2
S3150800051CE41A43461F1D1B4B4444994601339C461B
S3150800052CE24406E02B78013E237001350134002E97
S3150800053C14D000F035FBE31B4B45F3D94046514626
S3150800054CFFF7A6FF804600280ED0071D3C002B7827
S3150800055C013E237001350134002EEAD101201CBC62
S3150800056C90469946A246F0BD0020F8E75346070088
S3150800057C802208C7920051463800FFF719FF4346F8
S3150800058C1B68BAE7FF0100000123034A5B421360AC
S3150800059C024A13607047C046680100206C030020AD
S315080005AC10B5FFF7F1FF10BD134B70B516004A1EB8
S315080005BC04000D001B1A9A4201D9002070BDFFF7E2
S315080005CC09FFFF28F9D0601E4019FFF703FFFF2823
S315080005DCF3D00A4A630A5B02934206D02B00320018
S315080005EC21000748FFF77AFFE8E72B0032002100C5
S315080005FC0448FFF773FFE1E7FFFF0308002800082C
S3150800060C680100206C030020F0B5D6464F464646D6
S3150800061CC0B54E4B4A1E86B004000D001B1A9A42F2
S3150800062C07D90024200006B01CBC90469946A24661
S3150800063CF0BDFFF7CFFE8146601E4019FFF7CAFED4
S3150800064C4B460600FF2BECD0FF28EAD000234A467F
S3150800065C02930024042AE5D91628E3D88145E1D863
S3150800066C3B4B00251F009846052314373C009A4639
S3150800067C02E023780C349A4600F092FAD1455ED003
S3150800068C0135EDB2122DF4D101235B4299460523AF
S3150800069C3C009A46002502E023780C349A4600F072
S315080006AC7FFA564544D00135EDB2122DF4D101230B
S315080006BC5B429A460525002401E03D780C3700F08C
S315080006CC6FFAAE422ED00134E4B2122CF5D10023C7
S315080006DC49465246551AED18002303930123ED0A91
S315080006ECADB204910593002400F0D6FF002D0BD172
S315080006FC16E0802212019446049B01340193A4B29D
S3150800070C63440493A5420BD900F04AFA02A903A83C
S3150800071C01F06AF80028ECD0002400F0CFFF81E73E
S3150800072C0124FAE763001C19A40044446368CFE764
S3150800073C6B005D194346AD005B599A46BAE76B00E8
S3150800074C5D194346AD005B599946A0E7FFFF0308C0
S3150800075C6C20000800B5104A83B0136801200133D9
S3150800076C18D0916853688C46D16863448C461169D5
S3150800077C63448C46516963448C46916963448C4640
S3150800078CD26963449B185B4201AA0421034801936E
S3150800079CFFF70AFF03B000BD6C030020C028000851
S315080007AC0D4B18680D4B1B68C0180D4B1B68C018F1
S315080007BC0C4B1B68C0180C4B1B68C0180B4B1B68E2
S315080007CCC0180B4B1B68C0180A4B1B68C018434251
S315080007DC5841C0B27047C0460028000804280008D3
S315080007EC082800080C2800081028000814280008F7
S315080007FC18280008C02800080A4810B503680133F1
S3150800080C03D0FFF70DFE002808D00748036801330C
S3150800081C05D0FFF705FE431E9841C0B210BD012056
S3150800082CFCE7C0466C0300206801002000487047AE
S3150800083C0028000810B5FFF7B3FE10BD10B5FFF77A
S3150800084CB3FE10BD10B5FFF7DFFE10BD10B5FFF7F0
S3150800085CA7FF10BD10B5FFF7E9FF10BD10B5FFF7E0
S3150800086C79FF002801D0FFF7C7FF10BD0022054B02
S3150800087C05491A60596005219A601960034B1A607C
S3150800088C7047C04610E000E07FBB000070050020F2
S3150800089C0022014B1A60704710E000E0044B1B68FD
S315080008ACDB0303D5034A1368013313607047C0464C
S315080008BC10E000E070050020054B1B68DB0302D432
S315080008CC044B18687047034B1A68501C1860F9E7F4
S315080008DC10E000E070050020054B1B68DB0302D412
S315080008EC044B18687047034B1A68501C1860F9E7D4
S315080008FC10E000E0700500207047C04670B5094C42
S3150800090C80B22085FFF7D8FF0A300500802605E05F
S3150800091C00F046F9FFF7D0FF854202D3E3691E4281
S3150800092CF6D070BD00440040E12310B51B0288B018
S3150800093C01930C220023084C01A92000029303936F
S3150800094C049305920693079301F070F90122236824
S3150800095C1343236008B010BD0044004070B5040072
S3150800096C0D00402912D82800ADB2FFF7C7FF002D9D
S3150800097C0BD0013DADB20135651900F011F920789F
S3150800098C0134FFF7BBFFAC42F7D170BD8121024899
S3150800099C00F050F8E7E7C04644210008F8B5204DAA
S315080009AC0E002C78002C06D11E4BDA69920626D43A
S315080009BC00242000F8BD20241A4AD3691C4015D0FF
S315080009CC194C1A492378978CCA18577001330A7828
S315080009DCDBB223709A42EBD192B20131FFF7E8FCF5
S315080009EC00232B70237801243370E2E7FFF764FFAA
S315080009FC0F4B1B6864339842DAD92C70D8E79B8C5A
S31508000A0C0A4ADBB21370013B3F2BD1D8FFF754FFD0
S31508000A1C074B1860044B1C7001232B70C9E7C046A2
S31508000A2CB505002000440040B605002074050020DA
S31508000A3CB805002010B500F0B3F8FCE710B500F0C7
S31508000A4CA7F8012803D0094C2378012B00D010BD38
S31508000A5CFFF732FF064B1B68F533FF339842F6D384
S31508000A6C00232370FFF76AFCF1E7C046BC0500209B
S31508000A7CC00500200122054B10B51A70FFF71CFFA4
S31508000A8C034B1860FFF7DAFF10BDC046BC05002003
S31508000A9CC005002010B5FFF74DFC00F07DF8FFF7F8
S31508000AACE5FEFFF7C7FE00F00DF8FFF7E3FF10BDF4
S31508000ABC10B500F075F8FFF7F1FE00F013F8FFF724
S31508000ACCBDFF10BD10B500F06FF8FFF7A5FB0123AD
S31508000ADC034C2370FFF728FF0023237010BDC04674
S31508000AECC000002010B582B06B46104CD91D2000F2
S31508000AFCFFF7F0FB012811D06B462000D91DFFF734
S31508000B0C4DFF012801D002B010BD0022084B200071
S31508000B1C1A706B46D97900F065F8F4E7044B18702F
S31508000B2C6B462000D97900F05DF8E5E7C40500208E
S31508000B3CC00000207047C04670B50A4D06002B78D9
S31508000B4C0C00012B08D0002B03D1E1B23000FFF7C3
S31508000B5C05FF00F03FF870BDC9B2FFF79BFB2B7879
S31508000B6CF1E7C046C0000020054B40201B78013B2E
S31508000B7CDBB2022B02D8034A5B00985A7047C04670
S31508000B8CC00000207021000810B5FFF7EDFF10BD5E
S31508000B9C10B500F017F810BD10B500F061F910BDCE
S31508000BAC10B500F063F910BD00224321044B442014
S31508000BBC5A5400211A709A641A52997059707047CF
S31508000BCC04060020024B1878431E9841C0B27047A1
S31508000BDC0406002000214323014AD1547047C0461D
S31508000BEC04060020F8B503780500954CFF2B0CD0AD
S31508000BFC2278012A00D0F8BD3733DBB2352B00D961
S31508000C0C01E1904A9B00D3589F4600220125E370C8
S31508000C1CEF3B6270237162712570FFF7B5FFA07107
S31508000C2CFFF7A2FFE071FFF79FFF08224423000A93
S31508000C3C20726572A572E252FFF7FCFD4323E35C52
S31508000C4C012B05D04423E15E0029D4DD89B207E0E7
S31508000C5CFE2302220221E370EE3B23713433E25267
S31508000C6C01224323E01CE254FFF766FFC3E7FFF7B4
S31508000C7C8BFF6B78013898425DDDFF230122E37008
S31508000C8CBB3BE2526978002900D0C9E0FFF7E6FDC4
S31508000C9C0028D3D1FE230222E370CD3B23711333F4
S31508000CACE2524323E35C012BD2D04423E15AD7E723
S31508000CBCFFF744FBFF230122E370BB3BE252F0E74C
S31508000CCC4168A06CFFF7BEFD0028F3D1E2E70025CA
S31508000CDCFF232571E3706571FFF756FF072244233E
S31508000CECA071E57125726572E252DAE7FF23E370AB
S31508000CFC4768A66C002F00D19FE00025F7193378BA
S31508000D0C0136ED18EDB2FFF74BFFBE42F7D10022C4
S31508000D1C01230021E57123712D0E6271A2714333F3
S31508000D2C083221726172A572E252BAE7FFF72CFFFC
S31508000D3C6B7898426FDCFE230222E370DC3B23714E
S31508000D4C2233E252ADE7FFF71FFF6A789042F2DDD5
S31508000D5CA16C92B2201DFFF72BFBFF23A26CE3704C
S31508000D6C944644226B786344A3646B780133A3528C
S31508000D7C64E7FE23E3700023022223714433E25214
S31508000D8C8FE7FF236278E3700023627106222371D2
S31508000D9CA371E37123724433E25282E70023237072
S31508000DAC637087E7A66CFFF7EFFE6A1C411E3000DE
S31508000DBCFFF744FD002800D16CE7FF23E370FFF72B
S31508000DCCE3FEA36C01229C46442301386044A064CC
S31508000DDCE25266E7FF23E37043680122A3644423C7
S31508000DECE2525EE7FF23E370174B0721A364002347
S31508000DFC082223716371A37123726372A37244333D
S31508000E0CE171E2524DE7FE230222E370DE3B2371C9
S31508000E1C2433E25245E76968201DA1646A789AE78B
S31508000E2CAA1CA06CFFF70AFD002800D132E7A26CB9
S31508000E3C6B7894466344A36400E7002567E7C046CD
S31508000E4C04060020782100085022000810B500F08E
S31508000E5C3DF8024B18698004C00F10BD0008004805
S31508000E6C10B5642000F006F810BDC04610B500F0A9
S31508000E7C07F810BD014B18807047C0465006002075
S31508000E8C10B5FFF719FD0E4C236898420FD30D4B7E
S31508000E9C1A78002A0CD000221A7090232032DB050F
S31508000EAC9A62FFF709FD084B1B881818206010BDBD
S31508000EBC01321A7090231F32DB059A61F1E7C0469E
S31508000ECC54060020520600205006002090232022AB
S31508000EDCDB059A627047C0460121002210B5064B05
S31508000EEC494219611A61D960DA6099629A6201F00D
S31508000EFC27F8002010BDC0460010024010B50400AB
S31508000F0C00F0DCFCFA218900FFF7F6F800F08AFB02
S31508000F1C012000222100404200F050FB002010BDA9
S31508000F2C1021064A10B5136800200B431360FFF70F
S31508000F3CE5FF00F095FF002010BDC04600200240DA
S31508000F4CF0B501274A6A80261202C6463D0090462D
S31508000F5C0368B60098594C69334AA5401040424676
S31508000F6C0243E8433A4300B59A511C369A59024053
S31508000F7C9A51CA69002A3FD1103E9A59E400024098
S31508000F8C9A51CA688E881204324390261C19B600E8
S31508000F9CA2518A680E88120432439126B600A251D1
S31508000FAC81248A69A400002A22D11A5902401A51AE
S31508000FBC0A69002A16D18524A4001A59104018511A
S31508000FCC0A6A012A04D1872189005A582A435A5099
S31508000FDC8021012089005A5882435A50002004BCAB
S31508000FEC9046F0BD852080001A582A431A50E7E728
S31508000FFC1A592A431A51DBE7012AD1D18326B6009E
S3150800100C9A59E4002A439A510A688E881204324384
S3150800101C90261C19B600A2518A688E89120432438E
S3150800102C9126B600A251BBE7FFC0FFFF7047C0462A
S3150800103CF8B5051E00D17CE03D23C35CDBB2002B62
S3150800104C00D178E002213D23E9542B6801261A6861
S3150800105C8A431A601A6801390A431A60FFF73CFC7E
S3150800106C070004E0FFF738FCC01B0A2857D82B6882
S3150800107C5C683440F6D05A68164257D0AA69012AD9
S3150800108C5ED080211A688A431A60EA69012A00D15F
S3150800109C77E040211A688A431A602A6A012A00D125
S315080010AC6AE020211A688A431A606A6A012A5ED0A5
S315080010BC10211A688A431A60AA6A012A52D0082192
S315080010CC1A688A431A60EA6A012A46D004211A6801
S315080010DC8A431A60E968AA6801240A4329690A43FB
S315080010EC69690A43696801390A430121DA611A6890
S315080010FC8A431A60FFF7F0FB060004E0FFF7ECFBE7
S3150800110C801B0A2821D82B685A681442F6D15B68CA
S3150800111C23400BD12B643D230020EC5405E03D23E2
S3150800112C03220320EA54013BEC54F8BD04223D2368
S3150800113CEA540120F9E73C228354FFF777FF81E74D
S3150800114C80211A680A431A609FE703223D23EA5452
S3150800115C0022013BEA540320E7E704211A680A43F4
S3150800116C1A60B7E708211A680A431A60ABE7102118
S3150800117C1A680A431A609FE720211A680A431A60FC
S3150800118C93E740211A680A431A6086E7F8B54E4673
S3150800119C4546DE4657460368E0B59A6806000D00D4
S315080011AC520103D49A68120100D497E03C22B15C30
S315080011BC0220012900D18BE00121B1543C31725C2B
S315080011CCD2B2322A00D1C8E0622A00D1C2E0222A61
S315080011DC00D18CE0122272549A680024520106D46B
S315080011EC80229C6812052240544254410134C02086
S315080011FC01212201400090469A181758394011507F
S3150800120C316B8A4689688C46002900D092E01158C1
S3150800121C8C46514609684F055146C9680F436146C5
S3150800122C0F4317500F21894651460869494608400D
S3150800123C5146C2270861834648467F00D159434424
S3150800124C81435846D151D1590843D05151461800BB
S3150800125C49698930FF30016051468D338969FF33FE
S3150800126C1960C021012049005358484F0343535075
S3150800127CFFF732FB464B81469846326845490AE0E9
S3150800128C45480B4084466344581E8341DBB2002B09
S3150800129C0FD06B1C37D19368002CF1D0012C29D0B8
S315080012AC3E483B4084466344581E8341DBB2002BC0
S315080012BCEFD13D22B35CDBB2522B57D0722B52D0F6
S315080012CC422B4DD00123B35400223C230020F25468
S315080012DC3CBC90469946A246AB46F8BD9A68D200E5
S315080012EC00D563E704223D23C2540120F0E72032DF
S315080012FC725471E740460340294884466344581E95
S3150800130C8341DBB2C3E7002D06D0FFF7E5FA4B465F
S3150800131CC01A8542B1D2326803213D23F154002C00
S3150800132C27D1802193680B43936000223C2303202A
S3150800133CF254CDE711585746894651464968FF6815
S3150800134CC9008B46614639435F460F4349460F43EE
S3150800135C175067E7722272543EE7522272543BE7E3
S3150800136C203BB354B0E76223B354ADE73223B354EE
S3150800137CAAE791688023012C03D01B040B439360C6
S3150800138CD3E71B020B439360CFE7C046000001105E
S3150800139C0001000801000004FFFFFFFB0000FFEF3F
S315080013AC00FFFFF7F8B5CE4647463C2380B5150037
S315080013BCC25C06000C000220012A00D194E001222E
S315080013CCF254002900D093E00133F25C222A00D1B2
S315080013DCA9E0F25C422A00D1A5E0F25C622A00D1AF
S315080013ECA1E0F25C722A00D19DE0F25CD2B2322AFC
S315080013FC00D1CAE0522A00D1CDE0122A00D1C7E0AA
S3150800140C2222F254FFF768FA03278046326809E06D
S3150800141CD3683B4059424B41DBB2002B0BD06B1CBB
S3150800142C00D098E0002CF3D013693B4059424B414D
S3150800143CDBB2002BF3D1002C00D0A1E0736BD825BE
S3150800144C210157186D00785989468446042061464F
S3150800145C0840986000D08FE07859400D1860D82065
S3150800146C0125DA21400038584900400828408C46A6
S3150800147CD8600F2079580840614618617858494653
S3150800148C0004000E5118D8610800B930FF300768FF
S3150800149CBD311F750768FF313F0A5F7507681C6207
S315080014AC3F0C9F750068000ED87508681876086892
S315080014BC000A58760868000C98760968090ED976D9
S315080014CC002C38D12021D3680B43D3603D22B35C62
S315080014DCDBB2622B65D0722B66D0422B38D0B55452
S315080014EC00223C230020F2540CBC90469946F8BDC9
S315080014FC01290BD03D22B35CDBB2222B42D0422B06
S3150800150C4CD0122B14D03223B3547BE73D23F25C18
S3150800151C322A08D0F25C522A05D0F25C622A02D032
S3150800152CF35C722BE6D100223C230220F254DBE753
S3150800153C4033B35466E7202113690B4313613D22EC
S3150800154CB35CDBB2622B35D0722B30D0522BC6D1A2
S3150800155C1223B354C4E7002D06D0FFF7BDF9434652
S3150800156CC01A854200D351E703223D23F2540022C8
S3150800157C013BF2540320B7E77859C00858606EE768
S3150800158CB36B5CE76223B3543CE76222F25439E747
S3150800159C3032F25436E77222F25433E77223B354DC
S315080015AC30E73223B3549BE75223B35498E74223CC
S315080015BCB35495E72223B35492E7C04670B5002876
S315080015CC14DB164A03249446FF2283082040140091
S315080015DCC026C000890184400A4082409B006344AF
S315080015ECB6009D59A5432A439A5170BD0C4AFF244F
S315080015FC94460F230322C0B2034010402200C000B9
S3150800160C890182400C408440083B9B089B0063443C
S3150800161CDD6995432C43DC61E7E7C04600E100E051
S3150800162C00ED00E00A4A431E012093420ED8C02161
S3150800163C084A09485360036A09061B021B0A0B432E
S3150800164C0362002300209360073313607047C0467B
S3150800165CFFFFFF0010E000E000ED00E00C4B10B5BA
S3150800166CDA680023D20605D502210A4AD3690B4348
S3150800167CD3611023064AD16804220A4205D00124F4
S3150800168C04481343C1692143C161014AD36010BDA3
S3150800169C0020024058060020054B01201A69120644
S315080016AC04D50020034A5A60034A5A607047C0465C
S315080016BC0020024023016745AB89EFCD8021034A00
S315080016CC002013690B4313617047C0460020024083
S315080016DCF8B50500FFF700F9114C0700012601E0E3
S315080016EC6B1C12D1E3681E42FAD12023E26813421E
S315080016FC14D10B4BDA68D20603D4DB6800205B07DF
S3150800170C02D5FFF7ABFF0120F8BD002D04D0FFF77B
S3150800171CE3F8C01B8542E5D20320F5E7E360E8E76A
S3150800172C00200240F0B545465746DE464E46E0B523
S3150800173C9A4683B0294B019298461B7E04000D00ED
S3150800174C0220012B06D103B03CBC90469946A24612
S3150800175CAB46F0BD0123424621481376FFF7B8FF86
S3150800176C002833D1012C35D0022C35D00423013B6B
S3150800177CDBB25B0099460023AA1C914400269B46C3
S3150800178C18E05246DA401300424659460127154CD2
S3150800179CD16122699BB23A43226111482B80FFF72B
S315080017AC97FF2369BB43236100280FD102351036F6
S315080017BC4D450BD020235B42F318E2D52023524625
S315080017CC9B1B9A40019BF3401343DDE700234246DB
S315080017DC1376B8E70123CAE70223C8E758060020A0
S315080017EC50C3000000200240F0B54F464646D64688
S315080017FCC0B52F4F06003B7E89460220012B41D0EF
S3150800180C01233B7633682B48012B34D0FFF760FF56
S3150800181C002834D101234A465B421360B3687568C5
S3150800182CDB025B199D422AD20023234C98460AE018
S3150800183C80231B019C46726865449446B368DB0298
S3150800184C6344AB421CD9022243469246FB61236988
S3150800185C184813432361656123693E321343236198
S3150800186CFFF736FF52462369934323610028DFD0DE
S3150800187C4B461D6004E0FFF72BFF002807D001201C
S3150800188C00233B761CBC90469946A246F0BD04251F
S3150800189C4022094CF861236906482B4323612369C6
S315080018AC13432361FFF714FF2369AB432361E7E76F
S315080018BC5806002050C3000000200240014B18684F
S315080018CC7047C046C400002090220300D2059042FF
S315080018DC1CD02C4A904225D02B4A90422ED02B4A0B
S315080018EC904237D02A4A904240D02A4A0020934246
S315080018FC00D070478022284BD203996A01300A43DC
S3150800190C9A629A6A25490A409A62F2E78022224B21
S3150800191C9202996A01200A439A629A6A20490A40F5
S3150800192C9A62E6E780221C4BD202996A01200A4386
S3150800193C9A629A6A1B490A409A62DAE78022164B1F
S3150800194C1203996A01200A439A629A6A16490A404E
S3150800195C9A62CEE78022104B5203996A01200A43F9
S3150800196C9A629A6A11490A409A62C2E780220A4B1D
S3150800197C9203996A01200A439A629A6A0C490A40A8
S3150800198C9A62B6E70004004800080048000C0048B4
S3150800199C001000480014004800100240FFFFBFFF6B
S315080019ACFFFFFDFFFFFFFBFFFFFFF7FFFFFFEFFF4B
S315080019BCFFFFDFFFF0B5DE464E4657464546E0B517
S315080019CC0E688B46002E00D173E04B6800229C46AD
S315080019DC01235B42634498460AE059460969C36881
S315080019EC4D431C402C43C46033000132D34042D0D3
S315080019FC012393403340F7D01D0004685D43A1468C
S31508001A0C6C0064194F46E4432740B94667466F4352
S31508001A1CBA464F4651460F43414607600129DCD862
S31508001A2C81688A46594689686943894651462140E0
S31508001A3C8A464946574639438160C1688A4659469B
S31508001A4C09696943894651460C4049460C43614627
S31508001A5CC4600229C8D1FF2B1ED859466D43496963
S31508001A6C2C01641B4D43036A0132A3431D43330007
S31508001A7C0562D340BCD14346012B06D85A46436867
S31508001A8CD268B34356431E43466001203CBC90467D
S31508001A9C9946A246AB46F0BD59461B0A5B435B43C7
S31508001AAC49691D01ED1A4B43446AAC43234343620F
S31508001ABC9AE74B68013B9846DDE7C0460C23114A6A
S31508001ACC70B551680B40082B05D00C2B01D00E486D
S31508001ADC70BD0E48FCE75368C0225202134093426D
S31508001AEC0DD10A480F24074BD96A5D68214001318C
S31508001AFCFEF702FBAD0C2C4002346043E8E70248C3
S31508001B0CF0E7C0460010024000127A00006CDC02B6
S31508001B1C10B50400FFF7D2FF084A2060536808493D
S31508001B2C1B061B0FCB5CD84060605368054A5B05E7
S31508001B3C5B0FD35CD840A06010BDC04600100240B5
S31508001B4C582200086822000810B5031E18D1032075
S31508001B5C2C4C236B184002283DD0032846D001286C
S31508001B6C21D0FFF7ABFF626827491206120F8A5C71
S31508001B7C6368D0405B05254A5B0FD35CD84010BD23
S31508001B8C102813D1C0221F4C9202236B1A408023B3
S31508001B9C5B0513431E4A93422ED01E4A934225D008
S31508001BAC1D4A9342DDD1FFF789FFE8E70020122B87
S31508001BBCE5D1C022134C1203236B1A4090235B0504
S31508001BCC1343164A934217D0154A934209D0154A1D
S31508001BDC9342C6D1E7E7236A1840431E9841C003CF
S31508001BECCDE723689B07CAD50F48C8E723680020AA
S31508001BFC9B07C4D50C48C2E7206A8007C00FC003F0
S31508001C0CBDE7C046001002405822000868220008AA
S31508001C1C000002100000031000000110000008125A
S31508001C2C00000C120000041200127A0030B503688A
S31508001C3C85B004000D00DB072FD44B68C968026811
S31508001C4C0B4329690B43A9690B432D490A401343D6
S31508001C5C036043682B4A1340AA681343436083689E
S31508001C6C294A13406A6913438360284B98423FD02C
S31508001C7C274B984240D0274B984228D0264B98425F
S31508001C8C0ED0264B98420BD0254B984208D0254BA4
S31508001C9C984205D0244B984202D0002005B030BD9E
S31508001CAC01A8FFF735FF03980028F6D02968002904
S31508001CBCF3D08023AA691B029A420CD04B08181839
S31508001CCCFEF71AFA0004000CE0600120E6E7122081
S31508001CDCFFF73AFFE8E74B084000C018FEF70CFA86
S31508001CEC124B03400007400F1843E0600120D5E76C
S31508001CFC0020FFF729FFD7E71020FFF725FFD3E7CA
S31508001D0CF369FFEFFFCFFFFFFFFCFFFF0038014031
S31508001D1C0044004000480040004C00400050004081
S31508001D2C0014014000180140001C0140F0FF00009F
S31508001D3C014B18607047C046C40000200121114BA6
S31508001D4C11481A680A431A605A6802405A601A6897
S31508001D5C0E4802401A601A680D4802401A605A6802
S31508001D6C0C4802400F205A60DA6A8243DA621A6B10
S31508001D7C094802401A635A6B8A435A6300229A60CE
S31508001D8C7047C046001002400CB8FF08FFFFF6FE6D
S31508001D9CFFFFFBFFFFFFC0FFACFEF0FF10B5FFF720
S31508001DACBFF8012228490B68934313430B600B6851
S31508001DBC1A4243D08022254BD20219680A431A606C
S31508001DCC8022196852020A431A6080229202196804
S31508001DDC1142FCD05A681E491140A42292030A43A8
S31508001DEC0F215A60DA6A8A430E390A43DA6280226C
S31508001DFC196852040A431A608022144B9204196813
S31508001E0C1142FCD0F0215A688A435A605A68114923
S31508001E1C0A4003215A605A688A4301390A435A60B0
S31508001E2C0C220A494B681340082BFBD10A48FFF7CA
S31508001E3C7FFFFEF72FFEFEF73BFEFCE76A210748FD
S31508001E4CFEF7F8FDB6E7C046002002400010024037
S31508001E5CFF7FC2FFFFF8FFFF006CDC027022000850
S31508001E6CF0B50125334B8DB09A6980242A439A61C3
S31508001E7C9A69E4022A400592059A802259699202C7
S31508001E8C114359615969902611400491049958696E
S31508001E9C2027204358615969F6052140802403916F
S31508001EAC0399586924032043586159693000214025
S31508001EBC02910299D96900241143D961D9690A405A
S31508001ECC80210192019ADA6989040A43DA61DB698D
S31508001EDC06970B40009306A9009B0795089409944E
S31508001EEC0A94FFF767FD8023B7629B0106A912487F
S31508001EFC069307940A94FFF75DFD0C231E3F06A96B
S31508001F0C300006930797089409940A940B95FFF7E3
S31508001F1C51FDC0239B000693032306A90893074883
S31508001F2C0133079709940A940B93FFF743FD0DB0F9
S31508001F3CF0BDC046001002400008004800040048E6
S31508001F4C10B590242023E405A3621148FFF7BCFCC6
S31508001F5C1048FFF7B9FC2000FFF7B6FC0E4B0F49EB
S31508001F6CDA690F480A40DA61D9690E4A0140D96123
S31508001F7C59691140596159690B4A11405961012136
S31508001F8C5A6902405A619A698A439A6110BDC046D9
S31508001F9C000800480004004800100240FFFFFFFD3F
S31508001FACFFFFFDFFFFFFF7FFFFFFFBFF0D48854611
S31508001FBC0D480E490E4A002302E0D458C450043387
S31508001FCCC4188C42F9D30B4A0B4C002301E013605E
S31508001FDC0432A242FBD3FFF7B1FE00F011F8FFF76B
S31508001FECDDFEFEE700800020C0000020C8000020AF
S31508001FFC84220008C800002078060020FEE70000AE
S3150800200C70B500260C4D0D4C641BA410A64209D1C4
S3150800201C002600F019F80A4D0A4C641BA410A642B7
S3150800202C05D170BDB300EB5898470136EEE7B300FF
S3150800203CEB5898470136F2E77C2200087C22000808
S3150800204C7C22000880220008F8B5C046F8BC08BCFB
S3150800205C9E467047F8B5C046F8BC08BC9E46704705
S3150800206C00280008000800000500000000300008E1
S3150800207C00080000060000000038000800080000F0
S3150800208C07000000004000080008000008000000D7
S3150800209C004800080008000009000000005000086D
S315080020AC000800000A00000000580008000800009C
S315080020BC0B00000000600008000800000C0000007F
S315080020CC00680008000800000D00000000700008F9
S315080020DC000800000E000000007800080008000048
S315080020EC0F000000008000080080000010000000AF
S315080020FC00000108008000001100000000800108A3
S3150800210C0080000012000000000002080080000099
S3150800211C1300000000800208008000001400000074
S3150800212C000003080080000015000000008003086A
S3150800213C00800000160000002E2E2F2E2E2F2E2E7D
S3150800214C2F2E2E2F536F757263652F41524D434DAB
S3150800215C305F53544D333246302F756172742E638B
S3150800216C000000000800000000000000B00D000888
S3150800217C120E0008120E0008A00C0008120E000819
S3150800218C120E0008BC0C00087A0C0008CC0C0008CF
S3150800219CDA0C0008120E0008120E0008120E0008BF
S315080021AC120E0008120E0008120E0008120E000875
S315080021BC120E0008120E0008120E0008120E000865
S315080021CC120E0008120E0008120E0008120E000855
S315080021DC120E0008120E0008120E0008120E000845
S315080021EC120E0008120E0008120E0008120E000835
S315080021FC120E0008120E0008120E0008120E000825
S3150800220C120E0008120E0008120E0008120E000814
S3150800221C120E0008F80C0008380D0008520D0008BC
S3150800222CE00D0008120E0008120E0008120E000827
S3150800223CF00D0008120E00087E0D00088E0D000821
S3150800224CA80D00084F70656E424C54000000000043
S3150800225C000000000102030406070809000000003C
S3150800226C010203042E2E2F6D61696E2E6300000089
S3090800227CE500000863
S30908002280BD00000887
S30D080022840400000000127A00B4
S70508001FB91A
